:020000020000FC
:080000000C94DB090C94FB08D1
:040014000C946209DD
:04001C000C94CF0968
:04002C000C948E0999
:040038000C941A0901
:040048000C9460179D
:100050000C943017003B19EB0C3BA9EBD00005C307
:10006000000035C3E00082C30000BEC3420105AA00
:10007000000035AAAE0182AA0000B2AAC000059114
:10008000C6008291B201057800005978CC008278D0
:100090000000B278D400055F0000355FD800825FB1
:1000A0000000D65F1001054600004146BA018246B5
:1000B0000000CA462801052D0000412DC701051486
:1000C000426F6F74000044656D6F000043616C0007
:1000D0004E756D004C6564004275726E696E00006D
:1000E0004469616C00004F6E00004F66660031325B
:1000F000687200003234687200004865780044611C
:100100007465000042696E00526F6D004D696E00AB
:10011000506C617900004E6F726D00005265760080
:1001200046460000465200004E616D650000456481
:10013000697400005075736820546F2053746172A5
:100140007400475053004F6666002D3132002D3148
:1001500031002D3130002D3920002D3820002D3771
:1001600020002D3620002D3520002D3420002D3389
:1001700020002D3220002D312000302020002B3196
:1001800020002B3220002B3320002B3420002B3575
:1001900020002B3620002B3720002B3820002B3955
:1001A00020002B3130002B3131002B3132004453F1
:1001B00054004368726F6E6F00005265736574007F
:1001C0004A64520077007A0084008200860077003B
:1001D0007A007D007F007500750073008B008E0033
:1001E00090009200730075009700F800FA00750007
:1001F000555341004555000044656D6F2000420095
:1002000050004700FE120C135401E812F6125C0174
:10021000F113051464012F143F14680101173E12F5
:100220006C01331C3E127401481455147C011B13DD
:10023000251384012C1336138C013E1348139401AB
:1002400050135E139C015E146B14A40165137613A6
:10025000A8018413AD130000292AC71101802A2B9D
:10026000DB1102802B2CD41103802CB1CD110000A6
:100270002D2EC81118012E2FDB1110012F30D41193
:10028000080130B1CD1100003C3DC81118413D3E80
:10029000DB1110413E3FD41108413FB1CD110000A8
:1002A0004243C71105804341FC11048041C5FA1146
:1002B00000004540F211018040C4F01100004428C4
:1002C000FE1100003132C911200132B3E3110000E8
:1002D0003300E71100009281E7D6B4A392005140A9
:1002E0003625036251000CF80C46F846F8F80CF875
:1002F000FF0001FE0101FE01FEFE01FEFE01010103
:10030000FEFE01FE0101FE01FEFEFF0089018D01DE
:1003100091010B694F0B8C4FFF000B697F0B8C4FCA
:10032000FF000B694F0B8C7FFF009B01A001A50113
:10033000AA01AF01B4010B694F0B8C4F0BAF4FFFFC
:100340000B697F0B8C4F0BAF4FFF0B694F0B8C7FF3
:100350000BAF4FFF0B697F0B8C7F0BAF4FFF0B6910
:100360004F0B8C4F0BAF7FFF0B697F0B8C4F0BAF8D
:100370007FFFC301CA01D101D801DF01E601ED0110
:10038000F401FB0102020B694F0B8C4F0BAF4F0BBB
:10039000D24FFF000B697F0B8C4F0BAF4F0BD24F2F
:1003A000FF000B694F0B8C7F0BAF4F0BD24FFF0041
:1003B0000B697F0B8C7F0BAF4F0BD24FFF000B698C
:1003C0004F0B8C4F0BAF7F0BD24FFF000B697F0B96
:1003D0008C4F0BAF7F0BD24FFF000B694F0B8C7F05
:1003E0000BAF7F0BD24FFF000B697F0B8C7F0BAFE6
:1003F0007F0BD24FFF000B694F0B8C4F0BAF4F0B96
:10040000D27FFF000B697F0B8C4F0BAF4F0BD27F5E
:10041000FF003031323334353637383941424344C6
:1004200045460C0102030405060708090A0B0C01E6
:1004300002030405060708090A0B00000100010178
:100440000001FF01FF00FFFF00FF4A616E1F4665CC
:10045000621C4D61721F4170721E4D61791F4A7599
:100460006E1E4A756C1F4175671F5365701E4F6382
:10047000741F4E6F761E4465631F80FE80F2008DF0
:10048000FE8CF9009AFC99F700A6F8A5F400B3F4E5
:10049000B1EF00BFEEBAE500CAE6C7E200D4DED095
:1004A000DA00DDD5D9D100E5CBE1C800EDBFE4BA73
:1004B00000F3B4EEB200F7A7F3A600FB9BF69A0098
:1004C000FD8EF88D00FD80F18000FD73F87400FB57
:1004D00066F66700F75AF35B00F34DEE4F00ED410F
:1004E000E44600E536E13900DD2CD93000D423D0D4
:1004F0002700CA1BC71F00BF13BA1C00B30DB112DF
:1005000000A609A50D009A05990A008D038C080024
:100510007F037F0F0072037308006505660A0059A8
:10052000095A0D004C0D4E12004113461C00351B9C
:10053000381F002B232F2700222C2630001A361EAE
:10054000390012421B47000C4D114F00085A0C5B3A
:10055000000466096700027307740002810E8100BF
:10056000028E078D00049B099A0008A70CA6000CB8
:10057000B411B20012BF1BBA001ACB1EC80022D59C
:1005800026D1002BDE2FDA0035E638E20040EE45BA
:10059000E5004CF44EEF0059F85AF40065FC66F79C
:1005A0000072FE73F9FF7AEB7AD90080E883EB8959
:1005B000EB8CE88CE580D98CD900B5E4B5D200008D
:1005C000D2BBD5BEDBBEDEBBDEB8D2ACDEAC00003B
:1005D000E286E589EB89EE86EE83EB80EE7DEE7AAE
:1005E000EB77E577E27A00E580EB8000E04CD44CD5
:1005F000DD55DD430000B831AC31AC28B528B82555
:10060000B822B51FAF1FAC220000852182247C24B4
:10061000792179157C12821285158518821B7C1B25
:1006200079180047315331532E502B4D254D1F0063
:10063000224C1F4F1F52225528552B522B4F284C0E
:10064000224C1F491F46224328432B462B49284C46
:1006500000001D841A811A81148111841187148A63
:100660001A8A1D871D7B1A781478117B000021BE21
:1006700021AC000027BB2ABE30BE33BB33AF30AC49
:100680002AAC27AF27BB000049E449D2000053E45D
:1006900053D2FF0073EF76F27CF27FEF7FEC73E0D2
:1006A0007FE0008DE981E98AF28AE000AAE2AAD01F
:1006B0000000B0DFB3E2B9E2BCDFBCDCB9D9BCD624
:1006C000BCD3B9D0B3D0B0D300B3D9B9D900D0BC62
:1006D000D0AA0000E2B3D6B3DFBCDFAA0000DC89F9
:1006E000DC7700EE89E289E280EB80EE7DEE7AEB4A
:1006F00077E577E27A00D055D0430000E252DF552B
:10070000D955D652D646D943DF43E246E249DF4CBB
:10071000D94CD6490000AA2DAA1B0000B02DBC2D33
:10072000BC2AB927B621B61B00007B217B0F0083B2
:1007300018801B801E832189218C1E8C1B891883A5
:100740001880158012830F890F8C128C1589180060
:10075000492F491D00005B295826582652264F294B
:100760004F2C522F582F5B2C5B20581D521D4F20B1
:1007700000001E52215527552A522A4F1E432A4354
:1007800000002F52325538553B523B4638433243D6
:100790002F462F5200001187148A1A8A1D871D8444
:1007A00011781D780000238A237800001EBB21BE2B
:1007B00027BE2ABB2AB81EAC2AAC00002FBB32BE13
:1007C00038BE3BBB3BB82FAC3BAC000040DD43E048
:1007D00049E04CDD4CDA40CE4CCE000051DD54E017
:1007E0005AE05DDD5DDA5AD75DD45DD15ACE54CE84
:1007F00051D10054D75AD7FF76DF8ADF0079DF80E6
:10080000F30079F380DF0083DF83F30087F387DF72
:100810000076F38AF300ADD1B5D100B1D1B1E500D6
:10082000ADE5B5E50000D2ABDEAB00D6ABD6BF0080
:10083000DAABDABF00D2BFDEBF00DC76EE7600E0D6
:1008400076E08A00E576E58A00EA76EA8A00DC8AC4
:10085000EE8A00CA42DE4200CE42CE5600D356D7C0
:1008600042DB5600CA56DE560000A922B92200AD6E
:1008700036B122B53600A936B93600007514891490
:100880000079287D14812800851485280075288921
:100890002800432259220046364A224E3600512271
:1008A00051360055225536004336593600001D4258
:1008B000394200225626422A56002E422E56003237
:1008C0004232560036423656001D563956001177D0
:1008D0002377001477148B001877208B00188B2057
:1008E0007700118B238B000024AB32AB0027AB2F9A
:1008F000BF0027BF2FAB0024BF32BF0048D15AD161
:10090000004BD153E5004BE553D10056D156E500DD
:1009100048E55AE5FF007AEB7AD90080E883EB8955
:10092000EB8CE88CE580D98CD900E286E589EB89EF
:10093000EE86EE83EB80EE7DEE7AEB77E577E27A7A
:1009400000E580EB8000852182247C2479217915C3
:100950007C12821285158518821B7C1B7918001D5C
:10096000841A811A81148111841187148A1A8A1DAC
:10097000871D7B1A781478117BFF80EC8080FF8BB9
:10098000EC8080FF96EA8080FFA1E78080FFABE3E8
:100990008080FFB6DE8080FFBFD88080FFC8D18016
:1009A00080FFD0C98080FFD7C08080FFDDB6808007
:1009B000FFE2AC8080FFE6A28080FFE9978080FFA5
:1009C000EB8C8080FFEB808080FFEB758080FFE9FF
:1009D0006A8080FFE65F8080FFE2558080FFDD4A0D
:1009E0008080FFD7418080FFD0388080FFC8308072
:1009F00080FFBF298080FFB6238080FFAB1E8080F0
:100A0000FFA11A8080FF96178080FF8B158080FFE2
:100A100080158080FF74158080FF69178080FF5EDD
:100A20001A8080FF541E8080FF4A238080FF402967
:100A30008080FF37308080FF2F388080FF28418002
:100A400080FF224B8080FF1D558080FF195F8080D2
:100A5000FF166A8080FF14758080FF14808080FFFD
:100A6000148C8080FF16978080FF19A28080FF1D64
:100A7000AC8080FF22B68080FF28C08080FF2FC915
:100A80008080FF37D18080FF40D88080FF49DE80A2
:100A900080FF54E38080FF5EE78080FF69EA80800A
:100AA000FF74EC8080FF828080E67E808280FF8100
:100AB000808AE67E818180FF818095E47E818180CD
:100AC000FF81809FE27E818180FF8180A9DE7E811F
:100AD0008180FF817FB3D97E82817FFF817FBBD3FD
:100AE0007E82817FFF817FC4CC7E82817FFF817F78
:100AF000CBC57E82817FFF817FD2BC7E82817FFFDA
:100B0000807FD8B37F82807FFF807FDDAA7F828055
:100B10007FFF807FE1A07F82807FFF807FE3967FE1
:100B200082807FFF807FE58B7F82807FFF7F7EE5F5
:100B30008080827F7EFF7F7FE57680827F7FFF7F60
:100B40007FE36B80827F7FFF7F7FE16180827F7F99
:100B5000FF7F7FDD5780827F7FFF7E7FD84D818240
:100B60007E7FFF7E7FD24581827E7FFF7E7FCB3C72
:100B700081827E7FFF7E7FC43581827E7FFF7E7F84
:100B8000BB2E81827E7FFF7E7FB32881827E7FFFA6
:100B90007E80A92381817E80FF7E809F1F81817E50
:100BA00080FF7E80951D81817E80FF7E808A1B81F3
:100BB000817E80FF7E817F1B82807E81FF7E8175AA
:100BC0001B81807E81FF7E816A1D81807E81FF7E08
:100BD00081601F81807E81FF7E81562381807E819E
:100BE000FF7E814D2881807E81FF7E82442E817F21
:100BF0007E82FF7E823B35817F7E82FF7E82343C17
:100C0000817F7E82FF7E822D45817F7E82FF7F8273
:100C1000274E807F7F82FF7F822257807F7F82FFE7
:100C20007F821E61807F7F82FF7F821C6B807F7F3F
:100C300082FF7F821A76807F7F82FF80821A817F87
:100C40007E8082FF80821A8B7F7F8082FF80821C61
:100C5000967F7F8082FF80821EA07F7F8082FF80C0
:100C60008222AA7F7F8082FF808227B37F7F80825B
:100C7000FF81822DBC7E7F8182FF818234C57E7F91
:100C80008182FF81823BCC7E7F8182FF818244D33F
:100C90007E7F8182FF81824CD97E7F8182FF81812C
:100CA00056DE7E808181FF818160E27E808181FFCE
:100CB00081816AE47E808181FF818175E67E808109
:100CC00081FF828080BC7E808280FF818086BC7EA6
:100CD000818180FF81808CBB7E818180FF818092B9
:100CE000BA7E818180FF818098B77E818180FF817B
:100CF0007F9EB47E82817FFF817FA3B17E82817FD0
:100D0000FF817FA8AD7E82817FFF817FACA97E823B
:100D1000817FFF817FB0A47E82817FFF807FB39E31
:100D20007F82807FFF807FB6997F82807FFF807F78
:100D3000B9937F82807FFF807FBA8D7F82807FFF23
:100D4000807FBB877F82807FFF7F7EBB8080827FAA
:100D50007EFF7F7FBB7A80827F7FFF7F7FBA748038
:100D6000827F7FFF7F7FB96E80827F7FFF7F7FB62C
:100D70006880827F7FFF7E7FB36281827E7FFF7E7D
:100D80007FB05D81827E7FFF7E7FAC5881827E7FD7
:100D9000FF7E7FA85481827E7FFF7E7FA350818269
:100DA0007E7FFF7E7F9E4D81827E7FFF7E80984A80
:100DB00081817E80FF7E80924781817E80FF7E8060
:100DC0008C4681817E80FF7E80864581817E80FF8A
:100DD0007E817F4582807E81FF7E81794581807E14
:100DE00081FF7E81734681807E81FF7E816D478198
:100DF000807E81FF7E81674A81807E81FF7E816265
:100E00004D81807E81FF7E825C50817F7E82FF7E6D
:100E1000825754817F7E82FF7E825358817F7E82FB
:100E2000FF7E824F5D817F7E82FF7F824C63807F69
:100E30007F82FF7F824968807F7F82FF7F82466E4C
:100E4000807F7F82FF7F824574807F7F82FF7F82E9
:100E5000447A807F7F82FF808244817F7E8082FF10
:100E6000808244877F7F8082FF8082458D7F7F8064
:100E700082FF808246937F7F8082FF808249997FB4
:100E80007F8082FF80824C9E7F7F8082FF81824FA5
:100E9000A47E7F8182FF818253A97E7F8182FF8130
:100EA0008257AD7E7F8182FF81825CB17E7F8182AD
:100EB000FF818261B47E7F8182FF818167B77E80FE
:100EC0008181FF81816DBA7E808181FF818173BBC9
:100ED0007E808181FF818179BC7E808181FF103895
:100EE0003810100010006C6C480000000000002852
:100EF0007C28287C2800203840300870100064646A
:100F00000810204C4C002050502054483400303001
:100F100020000000000010202020202010002010C1
:100F20001010101020000028387C38280000001015
:100F3000107C101000000000000000303020000085
:100F400000780000000000000000003030000004C5
:100F500008102040000038444C54644438001030DD
:100F60001010101038003844041820407C00384419
:100F7000043804443800081828487C0808007C40DD
:100F800040780444380018204078444438007C04F9
:100F900008102020200038444438444438003844A5
:100FA000443C040830000000606000606000000005
:100FB00030300030302008102040201008000000A1
:100FC0007C00007C00002010080408102000384439
:100FD00004181000100038445C545C403800384459
:100FE00044447C4444007844447844447800384481
:100FF00040404044380078444444444478007C40B5
:10100000407840407C007C4040784040400038447C
:10101000405C44443C004444447C44444400381014
:1010200010101010380004040404444438004448EC
:101030005060504844004040404040407C00446C78
:101040005444444444004464544C444444003844AC
:101050004444444438007844447840404000384494
:101060004444544834007844447848444400384464
:101070004038044438007C10101010101000444414
:101080004444444438004444444444281000444404
:1010900054545454280044442810284444004444E0
:1010A00044281010100078081020404078003820A4
:1010B00020202020380000402010080400003808BC
:1010C000080808083800102844000000000000004C
:1010D0000000000000FC30301000000000000000A4
:1010E00038043C443C0040407844444478000000CC
:1010F00038444044380004043C4444443C0000006C
:101100003844784038001820207820202000000043
:101110003C44443C04384040704848484800100073
:101120001010101018000800180808084830404037
:1011300048506050480010101010101018000000A7
:101140006854544444000000704848484800000077
:101150003844444438000000784444447840000057
:101160003C4444443C04000058242020700000000B
:101170003840380438000020782020281000000073
:101180004848485828000000444444281000000003
:101190004444547C2800000048483048480000007F
:1011A000484848381060000078083040780018201F
:1011B00020602020180010101000101010003008BF
:1011C000080C080830002850000000000000387C9F
:1011D0007C7C7C7C38005A9A0E94221802E0109194
:1011E000F30210FD03E00093690001D00895E89A2E
:1011F0000895E89808950F930FB70F939460F882BD
:101200000F910FBF0F9118950F93F4BC05E005BD2A
:101210000FE707BD0F9108950DE70B8F0895FB8E23
:1012200002E005BB02E000936E00089500E0009329
:101230006E0008950F93F6BC78940FB70F931F9329
:101240000B8D002349F00A950B8F31F40091FD02BC
:10125000002311F49860FE8E0F8D000F1E2D4F9B02
:101260001127012B0F8F003849F40E8D0E15A1F0B8
:101270000FAD08600FAFEE8ECFDF0EC00F3721F03D
:101280000F3F51F40ED008C00E8D002329F090625C
:10129000FE8E0FAD077F0FAF1F910F910FBF0F9104
:1012A0001895C4DF01D0089500E800936D0004E0B4
:1012B00000936800089500E000936D0000E0009343
:1012C000680008950F930FB70F93F5DFA8DF0F9114
:1012D0000FBF0F91189504E00093810005E0009383
:1012E000890006E10093880013D0089508E017E014
:1012F000F8940C8F1D8F7894089500EF10E0F8CFCC
:101300001F930C8D1D8D012B09F00E2D1F9108953B
:1013100002E000936F00FC8EFD8E08950F93F09213
:101320008500F092840078940FB71F930F93BF93BA
:10133000AF93AC8DBD8D0A2F0B2B31F01197AC8F75
:10134000BD8F11F4E0929D020D85002329F00A95CE
:1013500011F490680E850D8709890A9511F490643F
:101360000FE0098BAF91BF910F911F910FBF0F91AC
:1013700018950F93F092B00007E00093B10003ECD2
:101380000093B30002D00F91089502E007BB02E082
:1013900000937000089500E00093700008950F938B
:1013A0000FB70F93F092B2000881039508830F9155
:1013B0000FBF0F9118950E94F4162227E0E0F1E08C
:1013C00014E0002721930A95E9F71A95D1F7CEE9A1
:1013D000D2E0FF24EE24E3949927882499240FEF88
:1013E0000F8F0AA708E208A30FE409A328E02F87BC
:1013F000EAE7F4E0E0930001F093010100E20BABB7
:10140000A0E4B1E0E4E5F0E016E3110F05910D93DF
:101410001A95E1F7E0929D020EE30D870E870FE02B
:10142000098B05E00B8BE9EDFAE0EDA7FEA701E8DB
:1014300000936400E9DE4FDF9CDF69D10E944B1806
:101440000E9474140E947E142FDF0E94C0190E9413
:101450000B1555D45ED40E94D8140E941D150E940D
:101460000D170090F702002011F00E9423170E9430
:101470003E180090E402002031F40090EE020020BB
:1014800011F40E9459190E94D8180E94F5184BD4E3
:101490006BD4EED20090E402002069F419811F930E
:1014A000A8D00E94CD181F9109810117C1F30A9598
:1014B000098374D290DE7894FAD4A6D20E94651A79
:1014C0000E945E1B0E94651A0E941D1792D095FF14
:1014D00025C09F7DE8E0FBE0EDA7FEA70E94AE12CD
:1014E00000E50E949812A8E4B1E00E948D12FEDE91
:1014F0008CD0EDD58CD709A10F3441F001DF00234A
:10150000B9F70E94A1120FE40E949812E9EDFAE0E7
:10151000EDA7FEA70FE409A3E0929D0293FF37C059
:10152000977FF88A0E944C160091F102073111F45E
:1015300002EC11C05EDE0E9499142DDF0091F102D1
:10154000083111F009EA07C00091F2020D3011F4E0
:101550000CEB01C00DEAD4D7C9DE4BD0B8D5D2D63A
:1015600008A1083239F0CCDE0023B9F7C2D7A3D7DF
:101570002ED74AD70091F102073121F006DF37DE7E
:101580000E949B14E0929D020E2D0E94531B00901E
:10159000F702002011F0A4D599CF90FD0E94671AA0
:1015A00095CFFF93EF93EDA5FEA50995EF91FF91E0
:1015B00008950F921F920F931F932F933F934F9372
:1015C0006F938F93BF93AF93FF93EF935F937F934B
:1015D00010D07F915F91EF91FF91AF91BF918F916B
:1015E0006F914F913F912F911F910F911F900F90ED
:1015F00008950090FC02002029F000917F040770FC
:1016000009F44AD3DAD024D0089510D121D0089516
:101610000F921F920F931F932F933F934F936F93AC
:101620008F93BF93AF93FF93EF935F937F93EDDF20
:101630007F915F91EF91FF91AF91BF918F916F91EA
:101640004F913F912F911F910F911F900F900895EF
:1016500092FF21C01D850E949B14011B19F00E31C1
:1016600008F406C00BA800FC02C098D101C0CED17E
:101670001091FD0210FF07C011FF0E94B11412FD6E
:101680000E94B71407C0A8A5B9A50A2E0B2A11F00D
:101690000E94B1149B7F97FF0AC0F8820E949E149B
:1016A0000BA800FC02C07AD101C0B0D19F7796FF91
:1016B00003C00E94C7199F7B94FF28C00B890A951D
:1016C00019F40E94B71405E00B8B0090EA02002089
:1016D00019F00E2D0E94531B9F7E0FAD01FF16C007
:1016E0001091EA020091E90210230091EF02102309
:1016F00051F00B81043039F4A0E3B1E0E0ECF1E00B
:1017000000EF0E9488190FAD0D7F0FAF0895209A4A
:10171000219A229A239A389A399A3A9A3B9A539A5A
:10172000549A559A5D9A5C9A0895582F580D5B0DFE
:101730005B9858B9529555B95C985C9A562F590DDB
:101740005C0D5B9A58B9529555B95C985C9A0895AE
:10175000562F580D5B0D5B9858B9529555B95C984A
:101760005C9A582F590D5C0D5B9A58B9529555B932
:101770005C985C9A0895382E462E880F880D8B0D44
:10178000660F690D6C0D0AD0839508D08A95639514
:1017900005D0839503D0642D832D08955B9888B977
:1017A000829585B982955C985C9A5B9A68B96295D6
:1017B00065B962955C985C9A08951F85A0E0B1E0D8
:1017C000ED91FD91BD90CD900E2E0F2A09F03AD0EB
:1017D0001A95B1F70888002041F4A0E2B1E015E0C5
:1017E0000FD0A4E3B1E013E016D0A0917F04B09134
:1017F00080041196A0937F04B09380045D9A0895AD
:10180000ED91FD91BD90CD900E2E0F2A09F082D062
:101810001A95B1F70895ED91FD91BD90CD900E2EE2
:101820000F2A09F070D01A95B1F70895A0E4B1E03D
:101830001AE1E6DF1E2DEFDF10917F041395109360
:101840007F040895BF93AF9385918823E9F38B308C
:1018500071F065914591442309F4F6CF4F3F89F02B
:1018600025912F934F9310D08F916F91F3CFC59007
:1018700005912B2D56D058D0B22E85918F3F09F06F
:10188000E4CFAF91BF910895DF01E5E9FBE0522F6E
:10189000561B08F45195042F081B08F401950517F1
:1018A00040F4E8EAFBE086276827862742272427BA
:1018B0004227481730F484274827842762272627A1
:1018C0006227442E481A522E561A08F451942224A4
:1018D00033246624621710F4639401C06A94481795
:1018E00078F05D980995250C3F1C722D720D7415CA
:1018F0003F041CF0660D24183F088395481790F7A5
:101900005D9AFD0108950DD00191002311F00CD0D6
:10191000FBCF089506D00591002311F005D0FBCF31
:1019200008954EED5EE008950F0107FD24C00152B9
:1019300008F15D98E02FFF27EE0FFF1FEE0FFF1F4E
:10194000EE0FFF1FE40FF51F68E06590882767FC26
:1019500012DF839566FC0FDF839565FC0CDF8395B2
:1019600064FC09DF839563FC06DF839562FC03DF7B
:101970006A9559F70F5D5D9AF00102D0B00E089597
:101980000A3311F408E009C0003811F404E005C07E
:101990000D3211F40AE001C00CE00895A8D71981B6
:1019A000139519831C3359F00A8D002311F0FA8E18
:1019B0002BC069D008A1007441F5D4D026C0906135
:1019C000F9821A8113951A831C339CF01FAD1260A3
:1019D0001FAFFA821B8113951B83183154F0FB82D1
:1019E00008A1007411F40E94BA151BA911FD5FD261
:1019F0000BC01BA911FD08C00E94131908A1007497
:101A000019F40E94F51853D233D0089570D70E857B
:101A10000D8719811A9519831F3F41F00A8C002008
:101A200011F0FA8E17C02FD09DD015C01BE319837B
:101A300090611A811A951A831F3F61F41BE31A8380
:101A40001FAD12601FAF1B811A951B831F3F11F43E
:101A500017E11B830DD008950E946E16002329F410
:101A60000E94D8180E94F51803D008950E94D81833
:101A700030D105D077D008950E94F518F9CF03D062
:101A800022D041D008950091F2020D3059F0EAE7DA
:101A9000F9E0098115E0019FE00DF11D8F01E8E0FB
:101AA000F1E05CC009810E94E616EAE2F3E009D1A8
:101AB000E8E0F1E000831183022FE2E7F3E001D1D7
:101AC000ECE0F1E04BC00091F2020D3059F0E6EA93
:101AD000FAE00A8119E0019FE00DF11D8F01E0E1BC
:101AE000F1E03CC00A810E94E616EAE2F3E0E9D0A8
:101AF000E0E1F1E000831183022FE2E7F3E0E1D0BF
:101B0000E4E1F1E02BC00091F2020D30B9F0E2EC1B
:101B1000FCE00A811CE00E94C5160F930B810E9415
:101B2000C516022F25E0029F1F91100D29E0129F7C
:101B3000E00DF11D8F01E8E1F1E010C00B810E9482
:101B4000E616ECE0F3E0BDD0E8E1F1E000831183BC
:101B5000022FE2E7F3E0B5D0ECE1F1E0008311837E
:101B6000D4D40895ACEAB1E03091F1023831A1F15A
:101B7000373111F4BED730C00B81363149F03431E2
:101B800039F40F01E2E2F4E0E00FFF1D0491F001EF
:101B90004ED00AE30D930A814AD00AE30D930981DE
:101BA00046D03091F102343151F400E80D9311E444
:101BB0000B810C300CF010E51D931DE41D9300907B
:101BC000FC02002049F0353111F0363129F41AE3D6
:101BD0001D9310E21D931D93FD9232D00CA900239A
:101BE00011F1ECEAF1E0A8EBB1E01CE001910D93FA
:101BF0001A95E1F71C970CA910E2013091F0023020
:101C000079F0033061F0053031F0043009F00BC099
:101C100013961D9306C017961D931D9302C013962D
:101C200013961D931D9308950CAB9CDF0895802F90
:101C30003091F102363111F452D701C04FD70895D7
:101C4000A8E3B1E0ECEAF1E0ED93FD9309D10D9347
:101C50000093E70209E40D930895A8E3B1E0FD9233
:101C6000FD92FD92FD9208950090FC02002069F023
:101C7000ACE3B1E0E4ECF1E0ED93FD930091E70219
:101C8000005A0D9309E40D930895ACE3B1E0FD9281
:101C9000FD92FD92FD9208950091F102053111F03F
:101CA000063171F4A4ECB1E00881043614F0045656
:101CB00000000BA800FE02C001950C59B8DFFD9290
:101CC0000895000FE00FFF1D05911491000F111FE3
:101CD0000895EDA9FEA90091F102083111F0073134
:101CE00029F40B810C3010F0EFA9F8AD0091F2024D
:101CF0000D3021F0E0930401F09305010895009167
:101D0000F102043110F0093118F004E10093F102FE
:101D100008950091F2020A3010F00F3018F00AE036
:101D20000093F20208950091F1020F93083189F0B7
:101D3000043131F0053139F0063129F0073101F075
:101D4000A4DF10DF08C00EDF8FDF05C09EDF0ADFD3
:101D500002C083DF9ADF0F9108950093F102E3DF61
:101D600038D6B7DFFFDE08950091F2020A3049F05D
:101D70000B3051F00C3079F00D3029F1E6E1F9E04B
:101D80000CC0E6EAF5E009C0E6EAF5E0EDABFEAB33
:101D9000E4E9F6E004C0E8EFF7E0EDABFEABEFAB53
:101DA000F8AFE6E2F1E009E7019304EB0193329624
:101DB0000BE6019304EB0193329607E8019304EBE1
:101DC00001935BD011C0E6E2F1E009E7019301E085
:101DD000019332960BE6019301E00193329607E8F6
:101DE000019301E001930BD043DE08950093F202CA
:101DF000BBDF0091F202E7D56CDF41DE0895EAE037
:101E0000F1E018EB108334961FEC108334961EE635
:101E10001083349615E81083349610E210833496BC
:101E200017E31083E6EEF2E0E0930001F093010186
:101E3000F0920401F092050119E101D00895A4E3A4
:101E4000B1E00090F902002041F4E7ECF1E0ED93FD
:101E5000FD9306D00D931D9302C0FD92FD9208954F
:101E600022270191002329F08BDD200FD0F70027D6
:101E700003C00FEF021B0695089506E0E8E0F1E0CD
:101E8000F192F192F19231960A95D1F7F0923401E4
:101E9000F092350111E9D3DFEAE7F4E0E0930001C5
:101EA000F093010116DF0895F092860402C0E092DB
:101EB0008604EFE9F2E029D0C5D058F066D00023BF
:101EC000B1F40091860400FD0E94A5157AD0EFDFE1
:101ED0000EC0E6D060F059D0002349F061D0002355
:101EE00031F40091860400FD0E94AF157ED0089564
:101EF0000091F402023039F00581085020F00830DA
:101F000010F488940895089408950091F402003024
:101F100059F0013009F1F0928104F0928304F092BB
:101F20008404F09282040895E3DFA8F312E0109392
:101F300081041BE0109382040F01E6EDF2E0E00F54
:101F4000FF1D0491F001102F12951F701093830450
:101F50000F70009384040895CBDFE8F2E0928104CF
:101F60001AE0109382040F01EFE6F1E0E00FFF1D8D
:101F70000491F001102F12951F70175E10938304C7
:101F80000F70075E009384040895EFE9F2E000C04B
:101F9000AFDF10F400270895102F0091F5020AC05A
:101FA000EFE9F2E000C0A4DF10F400270895102F3D
:101FB0000091F602112319F01A950695FBCF0170D6
:101FC0000895EFE9F2E000C093DF10F400270895D0
:101FD000102F1FD01091F502102B1093F502012F36
:101FE0000E94ED140E941F1A0895EFE9F2E000C06C
:101FF0007FDF10F400270895102F0BD01091F60208
:10200000102B1093F602012F0E94EF140E941F1A4A
:1020100008950E2D112319F01A95000FFBCF089586
:10202000E5EAF2E072DF0ED078F00090850400203F
:1020300039F0B9DF002341F4E5EAF2E0D9DF04C06A
:102040008894089555DF10F40894089504810330AE
:10205000D8F3B9F010918204011700F1A9F70381B8
:10206000109184040117D0F079F70281023010F04A
:1020700008940895F0928504013080F0E092850480
:102080000DC00381109183040117F0F239F402812D
:1020900010918104011710F408940895889408950C
:1020A00027DF10F40894089504811091820410171A
:1020B00060F0C1F7038110918404101730F091F79C
:1020C0000281023010F408940895889408950091D4
:1020D0007E04002321F00E94CF17F0927E04089521
:1020E00000917E04002349F000919D02002379F3C2
:1020F0000E946E16002359F701D00895F0927E04D5
:1021000033E6A8E3B2E00E94B217A8E3B2E0E4EC41
:10211000F2E20E94581100FF7CC002E00E944911C7
:102120000C91013409F075C0F0929D02E6D800913F
:10213000E902002311F404E074D001E00E94491187
:10214000C5D08987C3D08887C1D08F8309E00E941A
:102150004911BCD08A87BAD08B87B8D08C870985C3
:102160000090F802000D09871CF0083130F409C016
:10217000085E09870E94291104C0085109870E943E
:1021800024114EDF10F00E942E1109850B800015DE
:1021900049F408850A80001529F40F81098000158B
:1021A00009F409C009840B8208840A820F8009821D
:1021B0000E941319EA8E0C850E80001549F40B85D8
:1021C0000D80001529F40A850C80001509F409C05A
:1021D0000C840E820B840D820A840C820E944F199B
:1021E000EA8E0A8C0020A9F05FDEA4E2B1E0E2E012
:1021F000F2E00E948C190A2E0B2A49F005E0A00F8C
:10220000BF1D04E10D931296FD92FD9202C004E100
:1022100001D00895A4E2B1E0E2E0F2E00E94881962
:102220000895A4E2B1E0E2E0F2E00E948C190A2EE7
:102230000B2A49F4A4E2B1E002E0002E02E0102EE5
:1022400004E00E9467190895E5EAF2E00E94C215D1
:102250000895E5EAF2E00E94CA15089519851395DC
:1022600018311CF0F986F0DF112719870895E5EA87
:10227000F2E00E94E2151395011708F00027089577
:10228000FF93EF93E5EAF2E00E94E215EF91FF91F0
:102290000895A8E3B2E01127002E03940A9439F0C0
:1022A0000D9113950A3019F00C32C1F3F9CF08954E
:1022B0000D910590001521F40C32D1F70E2D01C0BF
:1022C00000270895244750524D432C000D911D9135
:1022D0000295007F1F70012B802F0E94D016089559
:1022E0000E94E4170090F702002019F40E942317BF
:1022F00002C00E942A170E240092F702002D0E94AD
:10230000F3140895E8E5F2E008A12FD008A30590A2
:10231000001611F03596FBCF95FF07C09F7D3196D3
:1023200005911491F80109951DC093FF1DC00591F9
:102330001CD0E6D00E947609329605911491002EA9
:10234000012A81F017FF02C06FDC0CC016FF08C025
:102350001F7B0F931F93D8011496C7D01F910F9125
:10236000D801B8D00E9476090895102F107811F086
:1023700090620F770895A0E2B1E004E30D9301E0CD
:102380000D9307E30D930DE20D931497089577D005
:1023900002C0F1DF90D098600895098103950C3355
:1023A00008F0002709830DC00A8103950C3308F05B
:1023B00000270A8306C00B810395083108F0002727
:1023C0000B8356DB08952FD70E94540F01C0F0D61F
:1023D00008E296D0F0922001F092210149DB0895A5
:1023E00017D4EFCF0C810AD4002311F41A951C8363
:1023F0009860089511D4E5CF13D4E3CF5CD04FD7C4
:102400000E94570F98600895F0D632DB0895E4E0FB
:10241000F2E009A10D3541F41091E002123009F407
:1024200003C00FE485D008950055002E000C000C69
:10243000000F000DE00FFF1D95FF06C09F7D05906A
:102440001590F001099517C093FF17C032960590BB
:102450001590FF93EF93F001099509A103950E35AF
:102460000CF00FE465D0EF91FF91A591B5910A2E84
:102470000B2A09F052D00E94760908950895A8E326
:10248000B1E0ECEAF1E008EB002E01E0102E0FEFD6
:102490000E946719AFA7B8AB0895A8EAB1E0E7ECCE
:1024A000F1E00CED002E01E0102E0FEF0E946719F5
:1024B000AFA7B8AB0895AFA5B8A90E94AA19FFA607
:1024C000F8AAFCAA0895ED91FD9112970FEF0E94D2
:1024D00088190895F8DFAAA3BBA30895AAA1BBA1F8
:1024E0000E94AA19FAA2FBA20895EDDFACA3BDA336
:1024F0000895ACA1BDA10E94AA19FCA2FDA2089555
:10250000977F08A3EBDFF5DF0895AAA1BBA10E9486
:10251000F919ACA1BDA16DD70895D5DFAEA3BFA3B6
:102520000895AEA1BFA10E94AA19FEA2FFA208951C
:10253000977F09A3F6DF0895AEA1BFA10E94F91904
:1025400008951091E002123011F4B5DF01D0089522
:1025500074D20ADC08958DD207DC0895088909AF8A
:102560006DD01091F1021DAF4FD00091E9020AAF7A
:1025700076D00091EF020BAF84D00091F2020CAF45
:102580002DD00BA80EAE92D00090F9020092E0027E
:10259000A4D00090FC020092DE027FD10090FA02EB
:1025A0000AAAF9AABDD0C8D00CE30090F702002017
:1025B00019F00091F802075B00939C021AD1009178
:1025C000F4020093DF0253D1F092E1027CD108952E
:1025D0000CAD03950F300CF00AE00CAF0CAD0A50B7
:1025E000E4ECF1E06EDBE4E5F1E021C00CAD10912C
:1025F000F202011711F0FADB17D008950DAD039523
:1026000009310CF004E10DAF0DAD0451EEECF1E039
:1026100058DBECE4F1E00BC01091F1020DAD0117B5
:1026200011F09BDB01D008950DE509A30895008307
:10263000118382DF089509AD0E2509AF09ADE8EDDC
:10264000F1E03FDBECE7F1E0F2CF09AD18890117CB
:1026500011F035D3E9DF08950AAD0E250AAF0AADB2
:10266000E4EEF1E02EDBE4E8F1E0E1CF0AAD109119
:10267000E902011711F059D3D7DF08950BAD0E25EC
:102680000BAF0BADE4EEF1E01CDBECE8F1E0CFCFFB
:102690000BAD1091EF02011711F050D3C5DF089573
:1026A0000EAD039504320CF000E20EAF0EAD0052F9
:1026B000ECEDF1E006DBE4E9F1E0B9CF0EAD1BA9EA
:1026C000011711F01DD3B0DF08950091E0020395CA
:1026D00003300CF000E00093E0020091E0020050B3
:1026E000E4EEF1E0EEDAE4EAF1E0A1CF0091E002FD
:1026F000023019F4F9AAD1DE06C01091F9020117CF
:1027000011F00BD391DF089509A9E7ECF1E0E00F98
:10271000FF1D0081039507FD00E200830DD00895A1
:10272000E7ECF1E00F010AA9E00FFF1DF082F001D4
:1027300097DB0093AA010895E7ECF1E0ACEDB1E07E
:1027400014E101910D931A95E1F709A9ECEDF1E07F
:10275000E00FFF1D0FE50083089509A9039509AB5C
:1027600003951AA901170CF00AAB0A9504316CF015
:10277000E7ECF1E00A9531F0E00FFF1D1081103217
:1027800009F4F6CF039509AB1EC0E7ECF1E00A951A
:1027900059F00A95E00FFF1D1191103229F41191A3
:1027A000103211F409AB0FC009A9E7ECF1E0E00F1A
:1027B000FF1D0081002311F400E20083B1DFBCDFC4
:1027C0000CE509A3089509A90093FA02E7ECF1E0EA
:1027D000E00FFF1DF082F092E602BDDE6CDE24DF2A
:1027E000089500919C02039506350CF00CE30093CC
:1027F0009C0220919C022C5306E411E0220F220F30
:10280000020F1F1DECE5F1E012CF00919C020C338A
:1028100091F009541091F702112321F01091F80260
:102820000117E1F00093F802E092F7020E94E4172A
:102830000E9423170CC0F092F8021091F7021123A6
:1028400069F0F092F7020E94E4170E942A170091A3
:10285000F702C9D00091F802C8D0E6DE08950091D1
:10286000DF02039503300CF000E00093DF020091DB
:10287000DF02EAEEF1E025DAE4E6F1E0D8CE0091FD
:10288000DF021091F402011711F070D2CDDE08952D
:102890000091DE020E250093DE020091DE02E8EDDB
:1028A000F1E00FDAE4E7F1E0C2CE0091DE02109130
:1028B000FC02011711F053D2B7DE08950091E10236
:1028C0000E250093E1020091E102E8EDF1E0F9D973
:1028D000ECE9F1E0ACCE0091E102002321F0EDD073
:1028E0000E940117A1DE0895569A5E9808950091FE
:1028F000E90200FF4E9A08955E98089557985F9AEE
:1029000008950AA50F3F71F4EAA6A091E202B091E2
:10291000E3020A2F0B2B31F400EF05D0A093E20263
:10292000B093E3020895A8E2B1E0EEEFF1E0F0D455
:102930000895FD8608950E850D8708950BA901FD64
:102940000895A8A5B9A50A2F0B2B21F40FEF03D0EA
:10295000A8A7B9A70895ACE2B1E0E0E0F2E0D8D4CE
:102960000895A8A5B9A5F6D4F8A6F9A608950A89E8
:102970000F3F61F00F01EAE3F4E0039507700A8B63
:10298000000FE00FFF1D85909490F00108950090D6
:10299000EF02002021F40090E5020A8AE8DF0895A2
:1029A0000A890093E5020FEF0A8B88249924089581
:1029B0000888002039F40091EF02002311F0F0DFC5
:1029C00001C0E5DF0895A9E01DC0A0E01BC0A6E09E
:1029D00019C0A8E017C0ABE015C0ACE013C0ADE073
:1029E00011C0A1E00FC0AEE00DC0AFE00BC0A5E08C
:1029F00001E008C0A0E106C0A2E104C0A3E102C05A
:102A0000AAE000C00090FD02002021F4BB2700BD19
:102A100016E0B1D10895ADEFB2E0E9EEF2E0AE1B01
:102A2000BF0B2A2FA0E0B0E011E0A5D10F3F09F4C1
:102A3000002701932A95C9F70895E7ECF1E000918A
:102A4000FA02002349F0202FAEE1B0E011E093D16B
:102A500001932A95E1F70CC0DF01E0E0FBE32BE0F6
:102A60002093FA0205910D932A95E1F7E092E60290
:102A700008950090FD020020F9F40090E602002085
:102A8000D9F40091FA02002341F400E20093C70157
:102A9000F092C8010E2D0093FA02202FA1E1B0E0C0
:102AA00000BD16E068D1AEE1B0E0E7ECF1E00191E5
:102AB00000BD61D12A95D9F70895ADEFB2E0E9EEF6
:102AC000F2E0AE1BBF0B2A2FA0E0B0E016E00FEF44
:102AD00000BD51D1F1922A95D1F7089571D18F930C
:102AE00082958F7079D18D938F918F7075D18D93E1
:102AF0000895EFE9F2E08381F1DF8DE28D93848127
:102B00000F01EAE4F4E08A95880F880FE80FFF1DB3
:102B100085918D9385918D9385918D938DE28D9384
:102B2000F00182E38D9380E38D938581D7DF089553
:102B3000EFE9F2E08281D2DF8AE38D938181CEDFFB
:102B40008AE38D938081CADF08951B8113951B83CF
:102B500018311CF0FB8216D0A2D365D308951B81D7
:102B60001A951B831F3F21F417E11B8313D097D3C2
:102B70005AD30895EFE9F2E005D00895EFE9F2E0C5
:102B800009D008955AD00E1521F461D00E1509F41C
:102B900067D0089503810A95038359F404810A9547
:102BA000048329F40CE0048305810A9505830AD087
:102BB00013830895FF93EF93EFE9F2E003D0EF91D1
:102BC000FF910895BF93AF930F930481AAE4B4E0FB
:102BD0000A95000F000FA00FBF1D1396FF93EF93F0
:102BE000FD011491EF91FF911C3121F405810370D7
:102BF00009F41DE10F91AF91BF910895EFE9F2E063
:102C000001D00895DFDF1395011708F0002708951C
:102C1000EFE9F2E012D00895EFE9F2E018D008955C
:102C2000EFE9F2E01DD00895EFE9F2E008C0EFE926
:102C3000F2E00FC0EFE9F2E015C003810395002335
:102C400019F0E0DF002309F40E2D038308950481B9
:102C50000395002311F00D3008F00E2D0483089524
:102C600005810395043608F0002705830895082F91
:102C70000C3310F48983089500270895082F0C332E
:102C800010F48A83089500270895082F083110F45E
:102C90008B83089500270895F1D179DE18E01F870E
:102CA00063D8089522D0E6D17BDEEF86E2EFF2E032
:102CB000E0930001F0930101089508890E25088B27
:102CC000002311F0EFDF01C0E7DF4EC00091F302F7
:102CD0000E250093F30294DE94D046C00BA9003277
:102CE00011F4002701C00E2D08950BA901FF03C0A8
:102CF0000EE30E870D8700E20BAB0E942C0D0895AA
:102D00001BA9102711FF05C01EE301FD12E01E875D
:102D10001D870BAB0E942C0D08950093F9026ADE0B
:102D200023D808950091E9020E250093E90200FDE1
:102D3000E3DD4BDE19C00091EF020E250093EF0298
:102D40000F9345DE0F9134DE0FC00091EA020E258D
:102D50000093EA0246DE08C00091FC020E250093B3
:102D6000FC024CDE0E94930E889408950093F402B6
:102D700032DE9DD80895A1BDB2BD119611FDFA9A1B
:102D80001FBBF999FECF00B50895222738E0000F48
:102D9000221F211710F00395211B3A95C1F70895C2
:102DA0000F921F920F938F9382958F700AE0809FEE
:102DB000002D8F918F70800F0F911F900F900895AD
:102DC000082F04D00295022B802F08951AE0DDDF32
:102DD0000A300CF00E2D08950F01E2E1F4E0E80F47
:102DE000FF1D8491F0010895A89504B7077F04BFE3
:102DF000009160000861009360000027009360006C
:102E00000895F894A895009160000861009360000F
:102E10000AE0009360007894089510E41093C400D1
:102E2000F092C500F092C00018E41093C10016E0C3
:102E30001093C200EC8AC8D008951091C1001069A7
:102E40001093C100089513E01093C40011E0109393
:102E5000C500089510E41093C400F092C5000895D1
:102E60000F930FB70F931F93FF93EF930F890F3FAC
:102E700079F00395EEEFF2E0E00FFF1D10811123D2
:102E800019F40FEFEC8A02C01093C6000F8B11C02B
:102E9000ED89FE890E2F0F2B31F0319614911123FD
:102EA00021F4FD8AFE8AEC8A04C01093C600ED8BE3
:102EB000FE8BEF91FF911F910F910FBF0F9118950E
:102EC0000F930FB70F931F932F933F93FF93EF939E
:102ED0002091C600088D302F03950F77198D0117AB
:102EE00031F40091F70200FDE0927E040EC0088FDD
:102EF000EEEFF3E0E30FFF1D208391602A3029F409
:102F00002091F70220FDE0927E04EF91FF913F9126
:102F10002F911F910F910FBF0F9118950F930C894F
:102F20000023E9F3FC8A8093C6000F91089590FF77
:102F3000FECF0F931F93FF93EF93188D098D882772
:102F4000011751F0EEEFF3E0E00FFF1D80810395D4
:102F50000F77098F011709F49E7FEF91FF911F9161
:102F60000F9108951127F894288D098DEEEFF3E065
:102F7000E00FFF1D808103950F771395131708F05D
:102F800011978D938A3029F0021781F79E7F8AE08E
:102F90008E93021709F49E7F098F78940895F89410
:102FA000288D098DEEEFF3E0E00FFF1D8081039582
:102FB0000F778A3019F00217A9F79E7F021709F4DC
:102FC0009E7F098F789408950FEF0F8BFD8AFE8AFC
:102FD00008950F939E7FF88EF98EF0927E040F91E4
:102FE00008950F93FF93EF930C890023E9F3FC8A74
:102FF000ED8BFE8B04910093C600EF91FF910F9132
:1030000008950F93FF93EF930C890023E9F3FC8A53
:10301000FF8AEEEFF2E00081002321F40FEF0F8B27
:10302000EC8A02C00093C600EF91FF910F910895C2
:10303000889490FD0894089508940C88002009F461
:10304000889408951F930F9319D003D00F911F9167
:1030500008951FE000E444D01EE001E841D011E0F3
:1030600001E13ED008951FE000E43AD011E001E113
:1030700037D008951DE000E833D008951DE0002703
:103080002FD00895000000000000000000000000A4
:10309000000000000895449A459A08953F9333270D
:1030A0003A9519F4E092E40217C0B1F06AD0EADF71
:1030B00002EA3FD0E7DF33D098F3012F3AD0E2DFC6
:1030C0002ED070F355D05DD003EA33D0DBDF27D0AC
:1030D00038F33CD0449A459A4BD0802F3F910895C5
:1030E0003F9333273A9519F4E092E40215C049D092
:1030F000C9DF0F9302EA1DD0C5DF11D00F9190F305
:103100000F93012F16D00BD00F9160F30F9311D0B6
:1031100006D00F9138F300002BD03F9108953C98D2
:10312000449A0894459AAEDF349B889445983C9A1B
:1031300008953F9338E0449A000F08F04498459A68
:10314000A1DF45983A95B9F73F9108953F933C9890
:10315000449A002738E0459A089494DF349B889479
:10316000001F45988FDF3A95B1F73C9A3F9108953B
:103170004498459A00000000449A00003C983D980D
:1031800008953C9A3D9A449A459A0000000044985C
:10319000000000004598000008958F9312E07EDF44
:1031A0008F77FEDD8C330CF0882789838F9108950B
:1031B0008F9312E073DF87FDA4DB8F77F1DD8C3313
:1031C0000CF08827898313E069DF8F77E9DD8C3382
:1031D0000CF088278A8314E061DF8F73E1DD88318A
:1031E0000CF088278B838F9108950F938F9315E0B0
:1031F00055DF8F73D5DD80320CF08E2D8C8317E078
:103200004DDF8F71CDDD882311F08D300CF08E2DC8
:103210008D8318E043DFC4DD84360CF088278E836D
:103220008F910F9108958091FD02882331F4898157
:1032300005D08A810DD08B8113D008958F93082FEC
:103240000C3320F48983BCDD12E04ADF8F910895AE
:10325000082F0C3320F48A83B3DD13E041DF089597
:10326000082F083120F48B83ABDD14E039DF08959B
:10327000C5DC002329F00C83802FA2DD15E030DFB0
:103280000895082F0D3020F48D839ADD17E028DF94
:103290000895082F8E8394DD18E022DF08950C81B5
:1032A000E7DF002309F4A1DF8D81EBDF8E81F1DF01
:1032B00008958827C3DF8827CBDF8827D1DF01E087
:1032C000D7DF81E0DEDF8827E4DF91DB0895BF935D
:1032D000AF93A2EFB1E016E02D913D91232B31F099
:1032E00018961A95C9F7EF91FF9111C0ED93FD93D0
:1032F000ED920D93EF91FF9101910D9301910D933B
:103300000D921D921A973297ED93FC9311970895A1
:1033100000241124DCDF08954F935F93AD01A2EFE9
:10332000B1E016E02D913D91022E032A61F02417A1
:10333000350739F42D913D912E173F0719F4149755
:1033400006C0129616961A9569F7AA27BB275F91B1
:103350004F9108950A2E0B2A69F0FF93EF93ED9198
:10336000FD9114960D911D9101931193189703D01F
:10337000EF91FF9108950AE0FD920A95E9F708950B
:1033800017E0A2EFB1E0F7DF1A95E9F70895A2EF91
:10339000B1E026E0BF93AF930D911D91012B21F079
:1033A00012972F9307D02F91AF91BF911A962A951C
:1033B00089F708950D911D9112962D913C913F3FF3
:1033C00019F03A953C9371F0322F3E253E9322231B
:1033D00011F0149601C012972D913D91D8012D93B3
:1033E0003D9306C01597FF93EF93B4DFEF91FF91E4
:1033F00008954A2F4B2B59F04D914E1741F44D91A2
:103400004F1729F40D931D9312960D931D93089554
:103410003DD1FE92FE9256D0AAEAB0E002C0A2E3ED
:10342000B0E011E0A8DC002349F00F3F39F0BF9372
:10343000AF93802F3ED0AF91BF91F3CF66C0E8ED40
:10344000FAE3AEEFB2E034D104D02ED1FD923AD0FF
:10345000089506E48091F50208D002E48091F60216
:1034600004D0089580E28D9308950D9338DBFADF40
:103470000895813624F08B3710F400E2801B089504
:103480000C94D10AD9DD10F0FBDFFCCF08950F9327
:1034900009818EE1080F0C330CF00C53C9DD28F0C4
:1034A000EFDF8981081721F0F9CF41DD0F912DC0A1
:1034B0002EC08F93E7DF8F9131DD0895FBE3E2DFCC
:1034C00090DD0895DFDF9DDD0895E2EEF7CF2FDD7B
:1034D000D0DF8835B9F4EEEAFAE3F1DFD8DFE9DFCF
:1034E000C8DFF3DF8154BCF38A31ACF7880FEAE719
:1034F000FAE3E80FFF1D05901590F001099510F40F
:10350000E0E9DCDFDDD0EA8E089588940895089420
:103510000895E2EAD3DF0895ECE29ED0B8F0B5DB7F
:103520000817A1F4D2DFEAE397D080F0A7DB0817F1
:1035300069F4CBDFEAE490D048F099DB081731F466
:1035400072DE0E94540F0E94380D38C00E94360D62
:10355000DECF0091EA02002321F02ADE46DE0E943F
:10356000380D94D0D2CFEAE577D0D0F0082F62DBC7
:103570000817B1F4AADFECE66FD090F0082F57DB04
:10358000081771F4A2DFEEE767D050F0082F4CDB8C
:10359000081731F484DE0E94570F0E94380D0EC0C8
:1035A00094DF0E943C0DB3CFB4DFE2EB55D040F086
:1035B000853030F48C5E082F0E94AD0E86DFA5CFDB
:1035C000A6CFA7DFE2EB48D038F0853028F4865F3D
:1035D000082F0E94F60EF2CF9ACF9BDFEAEB3CD089
:1035E00028F0833018F4082FC1DBE8CF90CF8DCFBF
:1035F00090DFE2EC31D030F0843020F4805E082F90
:103600007FDBDCCF84CFE0ED59DF7FCF56DA0E943D
:1036100001177BCFEAEC52DF1127A7ECB1E037DFCF
:10362000A8F047DF8D9313951431CCF38E9180323F
:1036300011F41A95D9F71196FC92112339F01093D1
:10364000FA02F092E6020E94AB125FCF0E94A8122B
:103650005ECF0E94011759CF31DF19DF2ADF88358D
:1036600009F455CF0CD0C8F3082F11DF22DF8835BD
:10367000C1F305D0D0F31AE0019F800D46CF80330F
:1036800020F08A3310F4805340CF41CF0F890F3F91
:1036900049F4AEEFB2E0E0E00AD0E2E108D0ECE0BD
:1036A00006D002D008950CC0E2EE01D00895FBE3ED
:1036B00005900D920020E1F711970895E7DF02C011
:1036C000AEEFB2E00F890F3F09F038C012DACADE60
:1036D0002FDAC8DE0091E902002311F48CE48D9307
:1036E0000091EF02002311F482E48D930091EA022D
:1036F000002311F086E58D930091F402023029F049
:1037000085E5002309F085E48D930091FC020023F8
:1037100011F08BE48D930BA9003211F086E48D93A8
:103720000889002311F083E48D939CDE92DE0DE482
:103730008091F3029ADEB8DFFD92C4DE089500277F
:10374000A7ECB1E005900D9203950020D9F70A95FA
:103750000093FA02F092F9020E94B40E08950E94BA
:103760007D0995FF02C09F7D4CDB0E94D10A0E941B
:1037700067100E9480090023A1F70895E0E2F1E0BC
:10378000A8EFB1E0A193B19309E601930DE2019393
:10379000ACDA2CD030D0E9EDFAE0EDA7FEA75CD092
:1037A000E0E0FBE3CCDF01D008950FD004D0D7DFF9
:1037B000089508E107C004E105C005E103C006E182
:1037C00001C007E10E94AD0E1BC00AE007C00BE07C
:1037D00005C00EE003C00DE001C00CE00E94F60E33
:1037E0000FC00E2D01C00027A0DA0AC0002701C0BB
:1037F0000E2D65DA05C0002701C00E2DB0DA00C01D
:103800000895ABA5BCA5A0E0B1E0EAE7F4E000E5CF
:103810007FDDABA7BCA70895ABA5BCA59BDDFBA630
:10382000FCA6089500E20E940A11089500E27BD8E8
:10383000089500E290D80895BEDF91DFC2DF8FDFE8
:10384000BCDF8DDFDADF8BDFD6DFB9DF88DFB3DF08
:1038500086DFAFDF84DF08950FE00B830AE20A837F
:103860000E94380D089501E00093FD0287DF2DDEF0
:10387000D6DDE2DFE2EAF9E362DFA7DF70DFA9DF8E
:103880006EDFA5DF6CDFA9DF6ADFE2EBF9E357DF6C
:10389000A2DF65DFD1DFEAEFF9E351DF90DF5FDF21
:1038A00094DF89DFE6E6FAE34ADF59DFE2EAF9E38B
:1038B00046DF55DFA2DF8BDF52DF9DDF82DF4FDF88
:1038C0008CDF4DDF88DF77DF4ADF83DF78DF47DF9C
:1038D00072DF7BDFEAECF9E332DF83DF40DF83DF97
:1038E0003EDFE8E0FAE32BDF3ADF82DF38DF7EDF1E
:1038F00036DFE0ECF9E323DF02E202DA30DF2FDF2C
:10390000F4D92DDF01E2FCD92ADF29DF03E2F8D95F
:1039100026DF25DFEAD9E6EDF9E311DF87DF1FDFD8
:103920001EDF03E00093FD0284DF19DF18DF01E0F2
:103930000093FD0277DF13DF12DF63DF10DF0FDF9D
:103940006BDFECE1FAE3FBDE05E00093FD02FA8AAF
:1039500006DF05DF01E00093FD02E0EEF9E3EFDEB4
:103960000E94AE12E8E0FBE0EDA7FEA7F8DEF7DE6E
:10397000E9EDFAE0EDA7FEA7EEE2FAE3E0DEEFDE26
:10398000EEE3FAE3DCDEEBDEE0E5FAE3D8DEE7DEE9
:103990000CDFE0EFF9E3D3DEE2DEE1DE0E940117A7
:1039A0000895596F7572204E616D65206865726566
:1039B000000042696E61727920436C6F636B000096
:1039C000506C6179204D6F6465004C454420436F15
:1039D0006E74726F6C005761726E696E677300006F
:1039E0004F6E2053637265656E204D656E750000E5
:1039F0005468616E6B20596F750042692D48657877
:103A000020436C6F636B000043616C696272617488
:103A1000696F6E2053637265656E00004275726E49
:103A2000496E2050726576656E74696F6E00416CE8
:103A3000736F20537570706F727465640000475027
:103A400053204E4D45412050617273696E670000EE
:103A50004461796C6967687420536176696E672088
:103A600054696D650000333020436F6D62696E618B
:103A700074696F6E730088940895851A9B165D169D
:103A8000B31A3B1DE11A7011081A331C291BAC161E
:103A900092166616D41A031BF81A851A061BA91A61
:103AA0008C1AED1AA5160A1B871A3B1DF71A436FCD
:103AB0006D6D616E6428422C432C442C462C472C9F
:103AC000482C4B2C4C2C4D2C4E2C502C522C532C27
:103AD000542C552C56293A004453542066697820BA
:023AE0000000E4
:103B0000447574636874726F6E69780056332E3131
:103B1000000020415652204F7363696C6C6F7363D1
:103B20006F706520436C6F636B2000003220646906
:103B3000676974206872733A20003220646967698B
:103B400074206D696E733A202000322064696769C1
:103B50007420736563733A202000322064696769BA
:103B60007420796561723A20202020003220646937
:103B7000676974206D6F6E74683A202020003220CF
:103B80006469676974206461793A202020202000EC
:103B90002043616E63656C2F54696D656F75740D9C
:103BA0000A00322064696769742076616C7565204B
:103BB000000028302D34293A000028302D32293ACF
:103BC000000028302D33293A00004E616D65200039
:103BD00028432932303038204A616E2064652052F3
:063BE00069650D0A0000FA
:00000001FF
